:100000000C94FA000C9417010C9417010C9417012E
:100010000C9417010C9417010C9417010C94170100
:100020000C9417010C9417010C94011A0C94D41A17
:100030000C9424150C9417010C9417010C941701BF
:100040000C9417010C9417010C9417010C941701D0
:100050000C9417010C94BC150C9417010C94170107
:100060000C9417010C9417010C9417010C941701B0
:100070000C9417010C9417010C9417010C941701A0
:100080000C9417010C9417010C9417010C94170190
:100090000C9417010C9417010C9417010C94170180
:1000A0000C9417010C9417010C941701B600B700BB
:1000B000162A0F082152BD00BE00A900AA000100A7
:1000C0000C0335006B006500790073000000140319
:1000D0006D0069006B006900790061003400310037
:1000E000380000000403090409023B00020100A0DB
:1000F000FA090400000103010100092111010001B6
:1001000022440007058103080001090401000103DE
:10011000000000092111010001227B000705820374
:1001200020000112010002000000084B4D010000F8
:10013000010102000105010902A10185020901A1D5
:100140000005091901290815002501950875018187
:10015000020501093009311581257F950275088155
:100160000609381581257F950175088106050C0A59
:1001700038021581257F950175088106C0C00501EB
:100180000980A101850319012AB700150126B700CE
:10019000950175108100C0050C0901A101850419A4
:1001A000012AA002150126A002950175108100C048
:1001B00005010906A101050719E029E71500250138
:1001C00095087501810295017508810105071900DF
:1001D00029FF150026FF00950675088100050819FE
:1001E00001290515002501950575019102950175F7
:1001F000039101C011241FBECFEFDAE0DEBFCDBFF7
:1002000011E0A0E0B1E0E0E4FBE302C005900D9254
:10021000A638B107D9F722E0A6E8B1E001C01D92E7
:10022000A333B207E1F70E94640F0C944C1D0C94A9
:100230000000823090F4611110C0453070F4E42F5A
:10024000F0E095E0899FE00DF11D1124EE0FFF1FF6
:10025000E455FF4F85919491089581E090E00895D1
:100260000E941901089581E008950E9433010895C4
:1002700081E008950E94330108950E943A01089593
:1002800008950E9440010895A6E0B0E0EAE4F1E09C
:100290000C94A81C49835A839E8330918D018981D7
:1002A0009A8131111AC03E81332399F0222389F0BB
:1002B0000E94D906182F682F89819A810E94BD0655
:1002C00069817A81812F0E94870D2696E3E00C9444
:1002D000C41C0E94CA06182FF3CF0E94D906698158
:1002E0007A81F1CFFC01262F408151816281738197
:1002F000848195810E9444010895CF93DF93D82F84
:10030000C92F61E00E9472016D2F7C2F0E94350180
:10031000DF91CF910895CF93DF93D82FC92F60E05D
:100320000E9472016D2F7C2F0E944101DF91CF91BD
:10033000089581E008950E9499010895CF93C82FF0
:100340000E948F058C2F0E949B012FEF84E39CE07D
:10035000215080409040E1F700C00000CF91089507
:1003600081E00E949E010E94E015089580E00E94B5
:100370009E010E94F11508950F931F93CF93DF9371
:100380008C0161E00E947201EC01B8010E943D0104
:100390008823B1F1B801CE010E949613882381F120
:1003A000B801CE010E94CA0F882351F1B801CE01D5
:1003B0000E949F0F882321F1F8018581882381F015
:1003C000CA35FCE7DF0739F178F4C130ECE7DE0726
:1003D000F9F0C330FCE7DF07C9F0C115DC4771F065
:1003E000C8010E9438010DC0CB35ECE7DE07B1F043
:1003F000CC35DC47A9F70E94DB0AF2CF0E94B0019E
:1004000080E0DF91CF911F910F9108950E94ED0A36
:100410000E94B601F5CF0E94E50AE2CF0E94E90AE8
:10042000DFCF0E9406150E94310208950E94350216
:100430000E940B15089581E008950895CF93DF93EE
:10044000D82F0E941B02C82F882319F08D2F0E94DD
:100450001D028C2FDF91CF91089508950E941E02F6
:10046000089580E00E942E0208950E94DC130E94ED
:100470002E020895CF930E94DC13C82F809188012B
:100480008C1779F0C09388010E94901560938901C0
:1004900070938A0180938B0190938C018C2F0E9422
:1004A0002E02CF910895ADE0B0E0E9E5F2E00C94C2
:1004B000A91C488759876A877B878C879D879111FC
:1004C0000E94180A1F8286E0FE013896DE0111960E
:1004D00001900D928A95E1F78D8181110DC02981DE
:1004E0003A814B815C816D817E818F810E945E09A2
:1004F0002D96E2E00C94C51CCE0101960E947D0170
:100500008111EDCFF5CFFC018481813021F4808110
:1005100091810E940B070895662329F00E943811EB
:100520000E94F91108950E948111FACFCF93C82F2C
:10053000882399F08CEF8C0F813A88F48C2F0E94DD
:100540006314882329F08C2F0E94A8140E94890A22
:100550008C2F0E94A0140E94890ACF91089580E2F6
:100560008C0F883048F4C77081E001C0880FCA95AD
:10057000EAF70E94F909EFCF8BE58C0F833038F44E
:100580002C2F2452330BC9010E940314E6CFE8E557
:10059000EC0FEB3150F4F0E0EE0FFF1FEB5EFE4F7F
:1005A000808191810E942914D8CF83E38C0F8331FD
:1005B000A0F661E08C2F0E948C02CFCF882381F1BE
:1005C0009CEF980F913A28F40E94A8140E94890A7F
:1005D000089590E2980F983050F4877091E001C030
:1005E000990F8A95EAF7892F0E94FF09EFCF9BE5C3
:1005F000980F933028F480E090E00E94031408954F
:1006000098E5980F9B3128F480E090E00E9429142F
:10061000089593E3980F933118F460E00E948C02E0
:1006200008951F93CF93DF93182FEB010E9496023A
:10063000209739F4812F0E94DE02DF91CF911F9124
:1006400008958FE99FE00197F1F700C0000021971E
:10065000EFCF60E070E0893311F460E570E00E9454
:1006600011030895882321F00E94F9090E94890A44
:100670000895882321F00E94FF090E94890A0895A5
:10068000A0E0B0E0E6E4F3E00C94A31C6C01D62FEC
:10069000C72FFC011581068102950F700E94EE099B
:1006A000E82E8823F9F0E12E1123E1F08C2F807FD2
:1006B000803461F080E28D0F8830F0F08C2F807EE6
:1006C000803221F4D230C0F00023B1F080911F02BB
:1006D00082FF12C082E00E94AE0A0E94EE0991E001
:1006E000E82EE926EC2FE295EF70C03CB0F5F0E083
:1006F000E25BF24E0C94931CE12CF4CF0C2F0F70A4
:10070000C03110F00295007F112399F0002359F0B9
:1007100080E28D0F883010F0D11107C0802F0E9429
:10072000F9090E94890A8D2F51C0802F0E940A0A60
:10073000F8CF8D2F0E94DE02002379F080E28D0F2A
:10074000883010F0D11104C0802F0E94FF0903C02F
:10075000802F0E94100A0E94890AEE2089F00E94D0
:10076000EA0980FD0DC0F60115820E94E4090E948D
:100770001A06C6010E9456050E94E4090E942A0634
:10078000CDB7DEB7E8E00C94BF1CFC2FFF70FF2E46
:10079000C07FC03219F0F29480EFF822DD2341F0DF
:1007A000D130D1F1112309F444C00023F1F0BBCFC3
:1007B00080911F0282FD15C0112359F0FF2029F0FE
:1007C0008F2D0E94F9090E94890A80E00E949602FA
:1007D000C4CF80E00E94DE02FF2009F4BECF8F2D3F
:1007E000B4CF112369F0011104C08F2D0E94320390
:1007F000B4CF013009F0B1CF8F2D0E94300AADCFB8
:100800000111ABCF8F2D0E9439038F2D0E943C0A1E
:100810008F2D0E941F0AA1CF112321F0063008F06E
:100820009CCFE3CF053008F098CF8F2D0E9439037D
:1008300094CF0023D1F3D93349F42FEF87EE93E01F
:10084000215080409040E1F700C000008D2F0E94B1
:10085000DE0283CF8C2F869586958370882369F07E
:10086000813009F07ACF8D2F9C2F9370111102C027
:1008700080E090E00E94291470CF8D2F9C2F937000
:10088000111102C080E090E00E94031466CF612F36
:100890008D2F0E948C0261CF8C2F8370811139C003
:1008A000111129C04D2F429546954770440F440FB2
:1008B0002D2F2F7030E0042E02C0220F331F0A9418
:1008C000E2F780E090E0D4FF09C08FE090E002C042
:1008D000880F991F4A95E2F780959095C695C69521
:1008E000C370822B932BC23071F0C33079F0C130CA
:1008F00039F00E94EA050E94DC130E942E022DCFDF
:100900000E94E105F8CF0E94F305F5CF0E94DE05B5
:10091000F2CF112361F1C0FFEECF4D2F42954695E6
:100920004770440F440F2D2F2F7030E0042E02C06B
:10093000220F331F0A94E2F780E090E0D4FF09C051
:100940008FE090E002C0880F991F4A95E2F78095EA
:100950009095C695C695C370822B932BC23069F0D3
:10096000C33071F0C13031F00E945506C4CF8230DF
:1009700010F2D3CF0E944C06BECF0E945E06BBCFC2
:100980000E940206B8CFCF70112339F08C2F0E943D
:100990001A068D2F0E943203AECF8D2F0E9439038D
:1009A0008C2F0E942A06A7CFD23F31F170F4D03F9E
:1009B000B9F0D13FB1F1112309F44EC0002309F47D
:1009C00048C08D2F0E94960296CFD33FE1F0D43FCE
:1009D00021F11111F3CF01114DC08C2F8F71E1CF97
:1009E000112341F0053008F086CF8C2F8F710E94C3
:1009F0003C0681CF0530F7CF8C2F8F711111D1CFED
:100A00000E941A0678CF112329F08C2F8F710E9433
:100A10000E0671CF0E9409066ECF80911F0282FDE3
:100A200006C08C2F8F71112309F4BBCFE9CF11239E
:100A300031F063E08C2F8F710E94900A5CCF81E0CF
:100A40000E94AE0A023008F456CF82E00E94AE0A3D
:100A500052CF8C2F8F71D4CF002309F4BECFD9335E
:100A600049F4EFEFF7EE23E0E150F0402040E1F7EA
:100A700000C000008D2F0E94DE023DCF0F931F9318
:100A8000CF93DF93EC01688179818D810E941807F3
:100A90008C010E9467060E94DD05B801CE010E940C
:100AA0004003DF91CF911F910F910895CF93DF9372
:100AB000EC018C81882399F0CE010E94BC01811148
:100AC00011C00E94EE09882351F08D81882339F0EE
:100AD00080911F0282FF03C082E00E94AE0ADF9174
:100AE000CF910895CE010E943E05CE010E948B0158
:100AF000F6CF80E090E00E94031480E090E00E9436
:100B000029140E94180A0E94890A0E9416120E9443
:100B1000F91108950E94B0140E94790508950E9469
:100B2000070A0E948A050895282F92959F70963093
:100B300091F060F4925F9F70923030F481E0203F3A
:100B400079F030F4283E30F080E008959A5FF3CFDA
:100B5000243FD1F7089581E0283EE0F3213FF9CF0B
:100B60000895FC018481882339F0808191810E945D
:100B70000B070E949405089580E00895A6E0B0E078
:100B8000E4ECF5E00C94A91C2696E2E00C94C51C5C
:100B9000A7E0B0E0EEECF5E00C94A91C2796E2E0AB
:100BA0000C94C51C08950E94D20508950E94D30597
:100BB0009093950180939401089508950E94D6051D
:100BC00008952091940130919501822B932B0E94DE
:100BD000D6050895209194013091950182239323A5
:100BE0000E94D605089520919401309195018227A5
:100BF00093270E94D60508950E94D20508950E9469
:100C0000FC0508950E94FF05909393018093920143
:100C1000089580E090E00E940206089521E030E00F
:100C2000A90102C0440F551F8A95E2F7CA010E942C
:100C30000206089521E030E002C0220F331F8A959A
:100C4000E2F78091920190919301822B932B0E9465
:100C50000206089521E030E002C0220F331F8A957A
:100C6000E2F7209530958091920190919301822333
:100C700093230E940206089521E030E002C0220F73
:100C8000331F8A95E2F78091920190919301822718
:100C900093270E94020608952091920130919301BA
:100CA000822B932B0E94020608952091920130918D
:100CB0009301822393230E940206089520919201BA
:100CC00030919301822793270E9402060895089588
:100CD0009B01677091E001C0990F6A95EAF763E0A4
:100CE000369527956A95E1F7220F331F220F331FA0
:100CF000FA01E20FF31F40E050E0682F70E08191AD
:100D0000DF0111979B01042E02C0369527950A94A6
:100D1000E2F7217021952827292328272C934F5F5C
:100D20005F4F4430510559F708959C01982F9770F3
:100D300083E0369527958A95E1F7220F331F220F1E
:100D4000331FFB01E20FF31F40E050E080E02191F0
:100D500030E0092E02C0369527950A94E2F72170FB
:100D60003327042E01C0220F0A94EAF7822B4F5F2B
:100D70005F4F4430510559F70895282F862F911160
:100D800008C0253030F4622F70E04EE851E00E9438
:100D900068060895282F892F911109C0253040F445
:100DA0006EE871E0822F90E00E949506089580E041
:100DB0000895A0E0B0E0EFEDF6E00C94A21C8C01E9
:100DC000E0909201F09093018091940190919501AF
:100DD000E82AF92ACFE0D0E0CC24C394D12CC60174
:100DE0000C2E02C0880F991F0A94E2F78E219F21D2
:100DF000892B49F4219798F7B12C8B2DCDB7DEB70D
:100E0000E9E00C94BE1CBC2EB8018C2F0E94930DFF
:100E1000019781F3F2CFCF93DF93D82FC92F0E9490
:100E2000D9066D2F7C2F0E94930DDF91CF910895ED
:100E30001F93CF93DF93162FD72F90918D01992376
:100E400041F0862F972F0E940B07DF91CF911F91C2
:100E50000895882381F0862F972F0E94D906C82FE6
:100E6000682F812F9D2F0E94BD06612F7D2F8C2F13
:100E70000E94930DEACF862F972F0E94CA06C82F93
:100E8000F4CF0F931F93CF93E0919601C7E0809129
:100E900097018E1304C0CF911F910F9108950E2FCB
:100EA00010E0CE9FF0011124E856FE4F20813181E1
:100EB000428153816481758186810E94C805F80151
:100EC0003196E770E4CF2091D0013091D10140916B
:100ED000D2015091D3016091D4017091D5018091DC
:100EE000D6010E94C80508958091D601803178F41A
:100EF0008091D501882359F0E091960120919701C6
:100F00003091D1014091D00157E02E1301C00895D6
:100F10006E2F70E05E9FF0011124DF01A856BE4FD6
:100F200014968C911497882361F111968C911197E6
:100F3000831327C08C91841324C015968C91159728
:100F400081111FC012968D919C91A091D201B091F8
:100F5000D3018A1B9B0B883C910598F48091D601A4
:100F60008F7080618093D601E256FE4F80818F7032
:100F70008061808380ED91E00E9456050E944107C8
:100F80000895FB013196E770C0CFE09196019091F2
:100F9000970127E0E91302C080E00895AE2FB0E08A
:100FA0002E9FF0011124E856FE4F3181361306C002
:100FB0003081381303C03581341304C0FD013196EC
:100FC000E770E8CF81E008958F929F92AF92BF9231
:100FD000DF92EF92FF920F931F93CF93DF93CDB7E2
:100FE000DEB72D970FB6F894DEBF0FBECDBF8C01D4
:100FF00086E0F801DE01189601900D928A95E1F7DE
:10100000F801E080F580A280B380848190ED892E84
:1010100091E0992E9091D40191111BC0882309F47D
:10102000FCC0FF2009F43DC1C8010E94B10588231E
:1010300009F437C187E0F801D40101900D928A9537
:10104000E1F7C4010E9483020E9474070E946307B3
:10105000E4C0D090D5012091D2013091D301A501F7
:10106000421B530BDD2009F4DBC0483C510508F05E
:10107000A6C0882309F4D1C09091D10191808091BC
:10108000D601803108F06BC0991228C09091D00130
:101090009E1124C0F1105DC08F7080618093D601D5
:1010A0000E94630780ED91E00E9456058091D60171
:1010B000F8018683F12C8F2D2D960FB6F894DEBFA4
:1010C0000FBECDBFDF91CF911F910F91FF90EF9099
:1010D000DF90BF90AF909F908F900895F11039C02E
:1010E00040E0692D8E2D0E94C50740E0692D8E2DB0
:1010F0000E94C507F82E8111DDCF888599850E9451
:101100000B07292F22952F70903450F49F702230B6
:1011100080F0992399F0F8019681903178F4CBCF43
:101120002A5F2F70223078F0C8010E945605FD2CEE
:10113000C2CF992319F0882309F4BDCF805E88308F
:1011400008F4B9CFF1CF803F08F4B5CF815F82308A
:10115000F7CF8091D60181608093D601ABCF9912F1
:1011600007C09091D0019E1103C0FF2009F479C0FF
:10117000C8010E94B105882309F493C0FF2009F437
:1011800090C08091D601803288F02091D0013091BA
:10119000D1013A832983BC82AB829091D4019D8393
:1011A0001E828F83CE0101960E94560587E0F801CA
:1011B000A0EDB1E001900D928A95E1F745CF9091B5
:1011C000D6019031A0F4488559856A857B858C8548
:1011D0009D850E94BE0580ED91E00E94560587E046
:1011E000F40111928A95E9F70E94630763CF88237F
:1011F000A1F02091D10181812813BACF8091D00133
:101200008E11B6CFF110B4CF9683C8010E94560557
:1012100087E0F40111928A95E9F7FF24F3944BCF0C
:10122000483C510508F041C08823B9F3FF20C9F1BB
:101230009091D101818198132AC08091D0018E11A3
:1012400026C08091D60180FD19C08031B8F0868318
:10125000807F803F39F08681982F907F905F8F70DC
:10126000892B8683C8010E94560587E0F801A0ED0E
:10127000B1E001900D928A95E1F7E8CE87E0F801A0
:10128000A0EDB1E001900D928A95E1F7C6CFC801BB
:101290000E94B10581118ACF8091D601816080932F
:1012A000D601C8010E945605B8CF488559856A8580
:1012B0007B858C859D850E94BE0591CFAEE0B0E018
:1012C000E4E6F9E00C94A81C288739874A875B87F5
:1012D0006C877D878E87CE0108960E94E40788235D
:1012E000B1F06C85662341F0288539854A855B8598
:1012F0007D858E850E94C80517E0809196019091AA
:10130000970189133EC02E96E3E00C94C41C87E03D
:10131000FE013896DE01119601900D928A95E1F753
:1013200020919701409196018C85882329F330E024
:10133000C90101968770992750E08417950799F0A5
:1013400097E0929FD001939FB00D1124A856BE4FF5
:10135000FE01319601900D929A95E1F780939701E5
:101360000E944107C9CF0E948F05109297011092E9
:10137000960187E0E0EDF1E0DF011D928A95E9F743
:10138000BBCF189FC001112488569E4F0E94E407CE
:10139000882309F4B8CFE09196011E9FF001112433
:1013A000E856FE4F208131814281538164817581ED
:1013B00086810E94C8058091960190E00196877011
:1013C00099278093960199CF8091DF018695869524
:1013D000869508958091DF01877008959091DF01CF
:1013E000977081E0911101C080E008958091EB0138
:1013F00008959091EB01982B9093EB010895982F0D
:1014000090958091EB0189238093EB0108951092D0
:10141000EB0108959091EA01982B9093EA010895C9
:10142000982F90958091EA0189238093EA0108958D
:101430001092EA01089508950E941B0A0895909160
:10144000E001292F2823222331F0809589238093DE
:10145000E0010E941C0A089508950E942C0A089534
:101460009091E101292F2823281729F0982B909398
:10147000E1010E942D0A08959091E101292F28236E
:10148000222331F0809589238093E1010E942D0A67
:1014900008958091E101882329F01092E10180E014
:1014A0000E942D0A08950F931F93CF93DF9300910D
:1014B000000110910101C091EB018091EA01C82B5C
:1014C000D091E101DD2331F00E944F1481110E947F
:1014D000490ACD2BF801C083C0910001D0910101D0
:1014E00048E050E067ED71E0CE010E94E41C892BDA
:1014F00059F088E0FE01A7EDB1E001900D928A95C8
:10150000E1F7CE010E94E913DF91CF911F910F9176
:1015100008950E94530A089508950E948C0A089520
:1015200090911F0292FF11C098E0899F90011124B1
:10153000622B6093DF010E941A068091DF0186957D
:10154000869586950E948D0A08950E941A06089530
:101550001092DF0180E00E948D0A08959091DF01D2
:10156000809589238093DF01282F277021110DC0DA
:10157000891759F090911F0292FF07C086958695B2
:1015800086950E942A060E94A80A089590911F023B
:1015900092FB222720F9281769F080FB92F990939B
:1015A0001F0280911E0290911F020E940E0B82E08A
:1015B0000E94AE0A089580911F0282FB882780F95D
:1015C00091E089270E94C60A089581E00E94C60A18
:1015D000089580E00E94C60A08956FEF7FEF80E0D3
:1015E00090E00E94361D089580E090E00E94021D68
:1015F0009C0181E0253E3E4F09F080E0089582E0A5
:1016000090E00E94FA1C089583E090E00E94FA1C8A
:10161000089584E090E00E94021D0895BC0184E0DA
:1016200090E00E94361D0895AB01BC018FE090E070
:101630000E942A1D0895AB01BC0183E190E00E9445
:101640002A1D089560E070E0CB010E941B0B0895F5
:1016500060E070E0CB010E94140B0E94220B089501
:10166000A8E0B0E0E6E3FBE00C94A91C65EE7EEF99
:1016700080E090E00E94361D60E082E090E00E94F1
:10168000181D81E090E0909395018093940161E0B2
:1016900083E090E00E94181D60E074E184E090E037
:1016A0000E94361D60E086E090E00E94181D60E018
:1016B00087E090E00E94181D40E050E0BA0188E009
:1016C00090E00E942A1D60E083E290E00E94181DD5
:1016D00060E08CE090E00E94181D60E08DE090E0FA
:1016E0000E94181D19821A821B821C821D821E8272
:1016F0001F82188648E050E067E170E0CE01019655
:101700000E94081D40E050E0BA018FE190E00E9485
:101710002A1D0E94280B2896E2E00C94C51C0E940A
:10172000300B0895682F8EE090E00E94181D0895F8
:10173000A6E0B0E0EEE9FBE00C94A71C0E94841543
:101740008C018091EC019091ED018017910779F067
:1017500019821A820E948415BC0149815A8180E055
:1017600090E00E9453021093ED010093EC01269645
:10177000E4E00C94C31C0E9490156093F3017093F5
:10178000F4018093F5019093F6016093EF0170935B
:10179000F0018093F1019093F20108950895089566
:1017A0000E94CE0B089508950E94D30B08958BE8F4
:1017B0009EE00E94790F0E94CF0B0E94D00B0895EB
:1017C00081E008950E94E00B08950E94E00B0895C7
:1017D000089508950E94E80B0E94E90B08950E9465
:1017E000F40A811102C00E948F0B0E94FF0A8093AD
:1017F000F7010E94090B90931F0280931E020E9422
:101800009C0F0E94040B90E00E94DE0580919201E3
:10181000909193010E94FF0508950E947B150E94FC
:10182000F00E0E94EF0B0E942D020E94D40B08952F
:10183000A6E0B0E0EEE1FCE00C94A41C0E94E20BF8
:1018400081110AC00E94980B0E9437120E943A022E
:101850002696E7E00C94C01C0E94FC0E1091EE014D
:1018600080E00E94950E181769F38091F70181FDC1
:101870000E949B0E0E94E50BD82E80E00E94950EE0
:10188000182F9091EE01891731F1E82EE92600E03A
:10189000FF24F3948F2D8E218823B9F0DD20A9F049
:1018A00009831A820E9484159C838B8381E08D8337
:1018B00091E08F2D8123811101C090E049815A81EF
:1018C0006B817C818D810E9453020F5FFF0C05307C
:1018D00009F71093EE010E94BB0BB6CF1F93CF9375
:1018E000DF930E94980DEC01811522E5920708F024
:1018F00053C0811540E5940708F0DDC0803E910596
:10190000F8F48D3C910508F0AEC0883A910580F45A
:10191000853A910508F099C08130910521F004972E
:10192000813A910550F4CE01DF91CF911F91089536
:10193000885A91094B9708F48BC0C0E0D0E0F3CFF0
:10194000811550E49507F8F4C11580E2D80708F036
:10195000CBC0C83ED10538F3CE019A9581159F4181
:1019600060F78D2F0E943C0E182FCE0199270E9400
:10197000980D212F30E0322F2227E901CC27DF718B
:10198000C82BD92BD0CF99270E94980DCC27DF7078
:10199000C82BD92BD06AC7CF803842E59407C8F549
:1019A000803652E5950708F067C0C03482E5D80755
:1019B000B0F08C2F86958695877020E2829FC001BB
:1019C0001124C37021E030E0A90102C0440F551F6B
:1019D000CA95E2F7EA01C82BD92BDC68A4CFC03244
:1019E00052E5D50708F041C08C2F8695869520E2F8
:1019F000829FC0011124C37021E030E0A90102C020
:101A0000440F551FCA95E2F7EA01C82BD92BDD68B0
:101A10008ACF803C52E5950760F48F71C03AD24579
:101A200008F03FC090E0982F8827EC01C46FD06A7F
:101A30007ACF805C9245809708F07FCFDC2FCC274F
:101A4000CC27DF71C06FD06A6ECFA497D0646BCF04
:101A5000C85AD0E0CC0FDD1FC55BDE4F0990D8819E
:101A6000C02DD46460CFD0655ECFCF71D0E0DC2FC5
:101A7000CC27C16FD06A57CF86958695877020E2B4
:101A8000829FC0011124C37021E030E0A90102C08F
:101A9000440F551FCA95E2F7EA01C82BD92BDA6823
:101AA00042CF0E943C0EC82FD0E0DC2FCC27CC27A1
:101AB000DF71D06238CF8F710E943C0E65E0D69501
:101AC000C7956A95E1F7CF70D0E0DC2FCC27282F9F
:101AD00030E084FF05C054E0220F331F5A95E1F730
:101AE000C22BD32BD0691FCF8D2F8F710E943C0E3C
:101AF000182FCE0199270E94980D212F30E0322F08
:101B0000222722273F71282B392BE901D2CF462FDC
:101B1000711106C0653020F460E00E943001089524
:101B200080E090E008950E94870D0E946E0C089559
:101B3000803E9105D1F1C8F48133910509F47FC04D
:101B400048F48932910509F46FC08A32910509F48D
:101B50007DC0089589339105E1F082389105C9F07F
:101B60008533910509F45BC00895843E9105D1F158
:101B700048F4823E910531F1833E910541F181EEB9
:101B800090E00895863E9105C1F1873E9105E1F10F
:101B9000089520911E022370211165C020911F021B
:101BA00023FF14C089E290E0089520911E0220FDD9
:101BB00043C030911F0230FF09C024FF4EC080E0B7
:101BC00090E0089520911E0222FDF7CF0895209104
:101BD0001E0222FD45C030911F0230FD44C024FF8B
:101BE000F5CFEDCF20911F0221FFF0CF80911E0293
:101BF00084FDE5CF87EE90E0089520911E0223FF3B
:101C0000E5CF24FDDCCFF6CF20911E0223FD2EC0B0
:101C100030911F0231FFE3CF84EE90E008952091D0
:101C20001E0225FFD3CFBECF20911E0225FD21C06D
:101C300020911F0223FFCACF89E390E008952091ED
:101C40001E0226FFC3CF8AE290E0089520911E0273
:101C500026FFBCCF81E390E0089583EE90E00895E5
:101C600082EE90E0089580EE90E0089586EE90E098
:101C7000089585E390E0AACF90911E0292FF10C0D4
:101C800041E0282F2471243009F040E031E0282F72
:101C90002871283009F030E0431711F02CE082273A
:101CA00093FF10C041E0282F2471243109F040E057
:101CB00031E0282F2871283109F030E0431711F066
:101CC0002CE0822730911F0230FF10C051E0282FF6
:101CD0002171213009F050E041E0282F287128308F
:101CE00009F040E0541711F029E0822731FF10C0BD
:101CF00041E0282F2171213109F040E031E0282F07
:101D00002871283109F030E0431711F029E08227CB
:101D100094FD877E089580E0089508950E948D0EB9
:101D2000089508950E94910E0895E82FF0E0EF5D68
:101D3000FD4F808108950895CF93DF93A1E8B1E02E
:101D400026E831E041E050E08D918F3FA1F0E82F8F
:101D5000E295EF70F0E061A18F70EA0102C0CC0F54
:101D6000DD1F8A95E2F7CE019C2F9095962391A3D3
:101D700092A1892B82A32A173B0731F7DF91CF91DC
:101D80000895CF93DF939C01C62FD0E085E0689F34
:101D9000F0011124EF57FE4F60E071E050E04191F7
:101DA0004F3FE1F0A42FA295AF70A05EB0E08C9100
:101DB00090E04F7002C0959587954A95E2F7817043
:101DC00081110CC0872F582B6F5F770F653039F763
:101DD000C20FD31F5883DF91CF91089580E0F3CFD6
:101DE0000E949C0E109221021092200281E00E941B
:101DF000210F0E948E0E0895A1E0B0E0E2E0FFE026
:101E00000C94A81C198260E0CE0101960E94C10EBC
:101E100090912002898121E0981310C020E041E0D8
:101E200061E272E080E292E00E94220F182F0E948D
:101E3000920E812F2196E3E00C94C41C8093200223
:101E4000EECF0895A0E0B0E0E8E2FFE00C94A31C20
:101E5000D82EE92EF62ED72F042FC22F222379F069
:101E600081E08093FA010E9484159093F901809398
:101E7000F80180E0CDB7DEB7E8E00C94BF1CC0905D
:101E8000FA01CC20B1F38091F8019091F9010E9400
:101E9000AD15059770F310E0A8016D2D7E2D8F2DE7
:101EA0009D2F0E94E41C892B41F0A8016D2D7E2DF1
:101EB0008F2D9D2F0E94F11CCC2D1092FA018C2F9A
:101EC000D9CF0E94180C08950E941D150E943F173B
:101ED0000E94D70B0E9459170E940D0C0E94661792
:101EE0000E946B170E94610F0E9485170E94EA0BE7
:101EF000F7CF909387018093860108950E94ED0AA1
:101F0000089580E00E94950E817008950E94FC0E55
:101F10002FEF86E791E0215080409040E1F700C02C
:101F200000000E94FC0E0E94810F882321F00E9475
:101F30007E0F0E94E01508950E94860F0895CF93AA
:101F4000DF93EB0186319C4719F50E94F6099D81CC
:101F50009923A1F08A7A91E0811101C090E09093D9
:101F6000FB01882349F085E30E94A0140E94890A9E
:101F700080E0DF91CF91089589E2F6CF8091FB0157
:101F8000882321F085E30E94A814F0CF89E2FBCFDB
:101F900081E0EFCFCF93DF93EC01FB0185818823B4
:101FA00009F4D2C09E0130572332310508F0B2C087
:101FB0000E94090B90931F0280931E02FE01E150C4
:101FC000F047E232F10520F4E65AF24E0C94931CED
:101FD00080911E02816080931E0293C080911F0237
:101FE000886080931F028DC080911E028260F3CFB3
:101FF00080911E028460EFCF80911E028860EBCF3B
:1020000080911F028160EDCF80911F028260E9CF35
:1020100080911E028061DFCF80911E028062DBCF43
:1020200080911E028064D7CF0E948F0580911E028E
:102030008068D1CF80911E028C60CDCF80911F022D
:102040008360CFCF80911E028E7FC5CF80911F020B
:10205000877FC7CF80911E028D7FBDCF80911E02EA
:102060008B7FB9CF80911E02877FB5CF80911F02F1
:102070008E7FB7CF80911F028D7FB3CF80911E02DC
:102080008F7EA9CF80911E028F7DA5CF80911E02E9
:102090008F7BA1CF0E948F0580911E028F779BCFEF
:1020A00080911E02837F97CF80911F028C7F99CFF2
:1020B00080911E0282FB992790F921E0922790FBE4
:1020C00082F990FB83F987CF80911F02982F90951A
:1020D00091708E7F892B90FB81F983CF90911E02A6
:1020E000892F8F7B96FF806476CF0E948F05909119
:1020F0001E02892F97FB87F980586DCF81E00E94DF
:10210000920B80911E0290911F020E940E0B0E9462
:102110008F0580E0DF91CF91089580E0F0CF90911E
:102120001E02892F8F7E94FF806155CF90911E02F1
:10213000892F8E7F90FF81604ECF90911F02892F53
:10214000877F93FF88604DCF81E0E4CF282F35EB68
:102150002303C001112497FF04C080589109892FDF
:10216000089580589F4FFBCF8091020280FF0DC0E1
:102170006091070170E0660F771F60387105C0F548
:1021800061157105B9F1862F089581FF07C060912F
:10219000070184E0689FB0011124EFCF82FF04C0E3
:1021A0006091070188E0F6CF809101028823E9F071
:1021B000909106016091070170E0891730F093E07B
:1021C000660F771F9A95E1F7D8CF869F9001879F7A
:1021D000300D112483E0220F331F8A95E1F7692F18
:1021E00070E0C9010E947F1CC8CF68E070E0CBCFCF
:1021F0008FE7089581E008958091020280FF0CC06E
:102200006091030170E07595679575956795611507
:10221000710561F1862F089581FF06C06091030169
:1022200070E075956795F3CF6091030170E082FDD2
:1022300015C0209100022223B1F09091020160911B
:10224000030170E0291750F4269FA001279F500D2D
:102250001124692F70E0CA010E947F1C603871054B
:10226000B0F28FE7089561E070E0D4CF81E0089587
:10227000E3E3E80FE331E0F5F0E0E458F24E0C94CC
:10228000931C0E94B41081958093060208950E94C9
:10229000B410FACF0E94B41081958093050208957E
:1022A0000E94B410FACF0E94FC1080930702089598
:1022B0000E94FC108195F9CF0E94FC1081958093BB
:1022C000080208950E94FC10FACF815D990B21E06D
:1022D00030E001C0220F8A95EAF780910402822B38
:1022E000809304020895809102028160809302022B
:1022F0000895809102028260F9CF80910202846089
:10230000F5CF409105028D3C59F48091060287FF7C
:102310000DC010920602442359F41092010208C025
:102320008E3C81F48091060218169CF3442381F0C0
:102330008091070290910802892B811159C0109257
:10234000000208958F3C41F447FFF0CF1092050240
:10235000809106028823E0CF803D19F41416B4F36F
:10236000E5CF90910702893D29F41916FCF61092E9
:102370000702DCCF8A3D19F497FFD8CFF8CF9091B0
:1023800008028B3D29F497FFD1CF10920802CECFDF
:102390008C3D19F41916CCF3C9CF9FE2980F9830F1
:1023A00090F4815D990B21E030E0B90102C0660F25
:1023B000771F8A95E2F7CB018095909104028923DB
:1023C00080930402B3CF8D3D31F4809102028E7F61
:1023D00080930202ABCF8E3D21F4809102028D7F6B
:1023E000F7CF8F3D09F0A2CF809102028B7FF0CF13
:1023F00008950E9484152091050230910602232B36
:10240000222321F08093FE019093FF012091070287
:1024100030910802232B222321F08093FC0190931A
:10242000FD0183E092E00E94F413089586E0E3E06A
:10243000F2E0DF011D928A95E9F7109201021092F5
:102440000002109202020895FC01828181110DC0E8
:10245000838181110AC08481811107C081E0958147
:10246000911101C080E08170089581E0FCCFA6E069
:10247000B0E0EDE3F2E10C94A61C86E0E3E0F2E0CC
:102480009E012F5F3F4FD90101900D928A95E1F790
:102490001092050210920602109207021092080292
:1024A0008B819C81892B8901882391F08091FE0189
:1024B0009091FF010E94AD159C018091010288233B
:1024C000C9F14091080150E04217530708F43FC09A
:1024D0008D819E81892B882399F08091FC019091B8
:1024E000FD010E94AD159C0180910002882309F432
:1024F00067C04091040150E04217530708F46EC0D2
:10250000B80183E092E00E94BB14811105C083E012
:1025100092E00E94241281110E94F91186E0F801D4
:10252000A3E0B2E001900D928A95E1F72696E5E0EE
:102530000C94C21C409109019AE0499FA00111240A
:102540004217530728F68F5F8093010202C08F3F26
:10255000D1F7FB80FF2059F00E94B41091E01F14C6
:102560000CF09FEF899F802D112480930502FC8041
:10257000FF2059F00E94B41091E01F140CF09FEF5F
:10258000899F802D11248093060280910502882363
:1025900009F49ECFF0900602FF2009F499CF0E9423
:1025A000A610811101C081E0809305028F2D0E9449
:1025B000A610882319F0809306028ACF81E0FBCF12
:1025C000409105019AE0499FA00111244217530749
:1025D00008F096CF8F5F8093000202C08F3FD1F743
:1025E000FD80FF2059F00E94FC1091E01F140CF0B8
:1025F0009FEF899F802D112480930702FE80FF208A
:1026000059F00E94FC1091E01F140CF09FEF899F7D
:10261000802D11248093080280910702882309F4F9
:102620006FCFF0900802FF2009F46ACF0E94A61035
:10263000811101C081E0809307028F2D0E94A610B6
:10264000882319F0809308025BCF81E0FBCF0F93C2
:102650001F93CF93DF93C42FD22FFC018581882352
:10266000C9F040930B020E94841590930A02809354
:10267000090280E28C0F883040F4C77081E001C00D
:10268000880FCA95EAF70E943203DF91CF911F911C
:102690000F91089510910B0214133CC08091090210
:1026A00090910A020E94AD15883C910598F5C0E210
:1026B000CD0F1D1741F180E2810F883040F4177073
:1026C00081E001C0880F1A95EAF70E943903C830EB
:1026D00020F0802F0E942903D8CF91E08D2F8770A2
:1026E00001C0990F8A95EAF7892F0E943203802F43
:1026F0000E942903D77081E001C0880FDA95EAF7BC
:102700000E943903C2CF802F0E942903C83008F0ED
:10271000BCCFF0CF80E28C0F883008F0B6CFC77006
:1027200081E001C0880FCA95EAF7EACF0F93FC0158
:10273000CB01E851FC47E730F10590F5E157F24E47
:102740000C94931C06E221EE41EE6AE17CE70E94C4
:10275000271380E00F91089507E225EE45EE6BE127
:102760007CE7F5CF06E221EE40EE68E17CE7EFCFB3
:1027700007E225EE44EE69E17CE7E9CF06E221EECF
:1027800042EE6CE17CE7E3CF07E225EE46EE6DE139
:102790007CE7DDCF08E221E045EE6EE17CE7D7CFB4
:1027A000FB018581811110920B0281E0D3CF9093C0
:1027B0001102809310020895E0911002F09111022D
:1027C000309729F00190F081E02D0995089580E07F
:1027D0000895E0911002F0911102309721F00280EB
:1027E000F381E02D09950895DC01E0911002F0914C
:1027F0001102309739F082E08C930680F781E02D4A
:10280000CD0109950895A3E0B0E0E9E0F4E10C946E
:10281000A91C9C0180910E0290910F0282179307D0
:10282000A1F030930F0220930E02E0911002F0917C
:102830001102309751F083E089833B832A8300841F
:10284000F185E02DCE01019609952396E2E00C94E6
:10285000C51CA3E0B0E0EFE2F4E10C94A91C9C01DC
:1028600080910C0290910D0282179307A1F0309392
:102870000D0220930C02E0911002F09111023097AA
:1028800051F084E089833B832A830084F185E02D25
:10289000CE01019609952396E2E00C94C51C409167
:1028A0000001509101019A012E5F3F4F485F5F4F39
:1028B00080E0F90190812F5F3F4F91118F5F4217A8
:1028C0005307B9F70895882371F0209100013091E2
:1028D0000101F9013296285F3F4F9191981729F035
:1028E000E217F307D1F780E0089581E008959C0195
:1028F000FC0132968FEF90E04191461751F08F3FE7
:1029000019F4411101C0892F9F5F9630A9F78F3FBD
:1029100009F40895280F311D87FD3A95F901628366
:1029200008959C01FC013296285F3F4F81918613E8
:1029300003C0DF0111971C92E217F307B9F708955E
:10294000682F80910001909101010E9477140895F1
:10295000682F80910001909101010E9491140895C7
:10296000E0910001F0910101329686E0DF011D92B5
:102970008A95E9F70895DC01FB0111969C91119766
:102980008181981322C012968C911297882319F096
:10299000928189131AC013968C911397882319F08A
:1029A0009381891312C015968C911597882319F07D
:1029B000958189130AC014969C91992321F081E096
:1029C0002481291303C080E001C081E08170089553
:1029D00008950E94E81408958F5F809312020E9468
:1029E000E914089583E0809312020E94E914089587
:1029F0000E94EC14089581E0809312020E94E91471
:102A000008950E94FB140895089508950E940515E5
:102A10000895089508950E94041508950E940915C7
:102A20000E94FC0E0E940A1580E00E94950E982FCD
:102A300081E0911101C080E0089585B7806885BF6D
:102A400085B7806885BF08951F921FB61F92112415
:102A50008F939F93AF93BF9380911302811113C003
:102A60008091220290912302A0912402B09125022C
:102A70004196A11DB11D8093220290932302A09341
:102A80002402B0932502BF91AF919F918F911F9027
:102A90001FBE1F90189580912A02843031F10E9448
:102AA00011021092130288E190E020E40FB6F8942E
:102AB000A895809360000FBE2093600083B7817F4C
:102AC000846083BF83B7816083BF7894889583B720
:102AD0008E7F83BF0FB6F894A895809160008861BF
:102AE00080936000109260000FBE08950E948F05D1
:102AF0000E941602089582E084BD93E095BD9AEF8E
:102B000097BD80936E0008952FB7F89480912202AC
:102B100090912302A0912402B09125022FBF089525
:102B2000A4E0B0E0E6E9F5E10C94A91C8FB7F894B5
:102B300020912202309123024091240250912502DB
:102B400029833A834B835C838FBF69817A818B8130
:102B50009C812496E2E00C94C51C9C014FB7F8942C
:102B60008091220290912302A0912402B09125022B
:102B70004FBF821B930B089578941F921FB61F922C
:102B800011248F939F93AF93BF93809122029091D2
:102B90002302A0912402B09125020196A11DB11D2E
:102BA0008093220290932302A0932402B0932502E3
:102BB000BF91AF919F918F911F901FBE1F9018954D
:102BC00087E797E7909301088093000888E19AE0EF
:102BD0000FB6F894A895809360000FBE90936000A4
:102BE000FFCF88E19AE00FB6F894A8958093600033
:102BF0000FBE90936000FFCF80911C02089508954E
:102C0000282FCB01BA0130912A023430E1F42F7021
:102C10002093E9002FEF3091E80035FD07C035ED36
:102C20003A95F1F7000021502111F5CF2091E800ED
:102C300025FF09C040E050E00E94FD178091E800A8
:102C40008E778093E8000895BC0143E050E082E075
:102C50000E9400160895BC0146E050E082E00E9408
:102C600000160895CF93DF93D82FC92F48E050E086
:102C7000682F792F81E00E94001688E0ED2FFC2F4D
:102C8000A4E1B2E001900D928A95E1F7DF91CF9136
:102C9000089580912902811109C00E9485190E941E
:102CA000E2198091E20084608093E200089510921E
:102CB000290208950E94FB1408956091260281E084
:102CC000611101C080E00E94F214089590912A02DF
:102CD00081E0943009F080E0609126020E94F814AF
:102CE000089542E061EC81E00E94011942E261EC4A
:102CF00082E00E94011990912A0281E0943009F04B
:102D000080E0609126020E94EC14089580912C02CC
:102D1000893089F148F4823009F4A0C0833009F485
:102D20005AC0813041F008958A3009F487C08B3051
:102D300009F46CC0089580912B02813A09F04AC0D1
:102D40008091E800877F8093E80080912F02909126
:102D50003002892B61F060E080E090E070E00E943A
:102D60004C188091E8008B778093E800089568E024
:102D700084E192E0F3CF80912B02813259F580916A
:102D80002F0290913002029728F58091E800877F0A
:102D90008093E8008091E80082FF18C09091F300D2
:102DA0008091F200029731F48091F100813011F0AE
:102DB000863021F48091F10080931C028091E8001C
:102DC0008B778093E8000E94351904C080912A0215
:102DD0008111E0CF089580912B02813AD9F780913B
:102DE0002F0290913002892BA9F78091E800877F0C
:102DF0008093E8008091E80080FFFCCF809114016F
:102E00008093F1008091E8008E77DBCF80912B02D8
:102E1000813201F780912F0290913002892BD1F6F7
:102E20008091E800877F8093E8000E9435198091A7
:102E30002D02809314010E948F05089580912B022A
:102E4000813241F68091E800877F8093E8000E94FC
:102E5000351980912E0280931D02089580912B02D6
:102E6000813A09F0B7CF8091E800877F8093E8002E
:102E70008091E80080FFFCCF80911D02C1CF84B714
:102E8000877F84BF0FB6F894A89580916000886111
:102E900080936000109260000FBE80E890E00FB653
:102EA000F89480936100909361000FBE0E94011519
:102EB00008950E9485190E94E219E2EEF0E08081F7
:102EC0008460808378940E94651C08958AE091E074
:102ED0000E94D713089580912A02853031F48091A1
:102EE0002A02853019F00E94761508950E944B152C
:102EF0000E940E15882399F380912802882379F384
:102F00000E94E7170E948F05EACF08959A01409129
:102F10003102509132020E948E170895AC01CB010C
:102F2000D901252F332723303105E1F058F4213022
:102F30003105C9F122303105D9F180E090E020E07F
:102F400030E01EC02132310521F122323105A9F7CE
:102F5000892BC1F16130710581F78BE790E025E3A2
:102F600031E00EC0CA019927413069F082309105E5
:102F700069F0E4EEF0E0892B01F7849190E09F0185
:102F80002D933C930895EEECF0E0F7CFE0ECF0E009
:102F9000F4CF892B91F06130710579F689E090E0EA
:102FA00023E131E0EDCF82E190E023E231E0E8CFB0
:102FB0008BE390E028EE30E0E3CF89E090E02AEF69
:102FC00030E0DECF84E490E020EB31E0D9CF80E147
:102FD00089BD82E189BD09B400FEFDCF8091D80092
:102FE0008F7D8093D8008091E00082608093E00024
:102FF0008091E00081FDFCCF0895AF92BF92CF9207
:10300000DF92FF920F931F93CF93DF936C01EB013D
:103010008A010E945419F82E811123C0011511054F
:1030200039F0F80180819181C81BD90BC80ED91ED7
:10303000A12CB12C2097A9F08091E80085FD22C039
:103040008091E8008E778093E80001151105A1F0CA
:10305000F801808191818A0D9B1D9183808385E099
:10306000F82E8F2DDF91CF911F910F91FF90DF9060
:10307000CF90BF90AF9008950E9454198823E1F239
:10308000F82EEFCFF60181916F018093F100219727
:10309000FFEFAF1ABF0ACECFFC019B018091310236
:1030A000909132028617970718F0672B61F0C901DB
:1030B00040E0009771F441110CC08091E80082FF5C
:1030C00035C080E008958091E8008E778093E80015
:1030D000EECF20912A022223A9F12530A9F12091D7
:1030E000E80023FD2DC02091E80022FDE6CF2091CD
:1030F000E80020FFDECF3091F3002091F20000972E
:1031000019F02830310558F041E02830310509F038
:1031100040E02091E8002E772093E800CACF41914B
:103120004093F10001972F5F3F4FE9CF80912A0232
:10313000882341F0853041F08091E80083FFBDCFC6
:1031400081E0089582E0089583E00895FC019B01E9
:1031500080913102909132028617970718F0672B01
:1031600061F0C90140E0009771F441110CC08091F9
:10317000E80082FF36C080E008958091E8008E77F5
:103180008093E800EECF20912A022223B1F125306E
:10319000B1F12091E80023FD2EC02091E80022FD2E
:1031A000E6CF2091E80020FFDECF3091F3002091A0
:1031B000F200009719F02830310558F041E028302E
:1031C000310509F040E02091E8002E772093E800D7
:1031D000CACF44914093F100319601972F5F3F4F42
:1031E000E8CF80912A02882341F0853041F0809118
:1031F000E80083FFBCCF81E0089582E0089583E07A
:103200000895982F973028F08F708093E90081E01F
:1032100008959093E900242F762F50E0981731F00D
:103220007091EC002091ED005091F00021FD02C062
:103230009F5FE8CF3091EB003E7F3093EB00309101
:10324000ED003D7F3093ED003091EB003160309325
:10325000EB007093EC002093ED005093F000209170
:10326000EE0027FDE5CF80E0089580912B0287FFD7
:1032700013C08091E80082FF06C08091E8008B7740
:103280008093E80004C080912A028111F2CF089552
:1032900080912A028823D9F38091E80080FFF8CF3B
:1032A0008091E8008E77ECCF2091E4003091E5002A
:1032B00095E6A9018091EC008170882331F080911E
:1032C000E80080FF06C080E008952091E80022FD1C
:1032D0001BC080912A02882391F0853091F0809163
:1032E000EB0085FD10C02091E4003091E50042170D
:1032F000530701F391509111DCCF84E0089582E0EF
:10330000089583E0089581E008950E94F4190E94D1
:10331000FC19E0EEF0E0808181608083E8EDF0E070
:1033200080818F77808319BCA7EDB0E08C918E7F70
:103330008C9380818F7E80831092290208950F9351
:103340001F93CF93DF930E94F4190E94FC19C8EDDC
:10335000D0E088818F77888388818068888388819E
:103360008F7D888319BC10922A0210922602109237
:1033700028021092270200EE10E0F80180818B7F76
:10338000808388818160888342E060E080E00E94E1
:103390000119E1EEF0E080818E7F8083E2EEF0E0C3
:1033A000808181608083808188608083F801808152
:1033B0008E7F8083888180618883DF91CF911F9188
:1033C0000F910895E8EDF0E080818F7E8083E7ED36
:1033D000F0E080818160808384E082BF81E080931F
:1033E00029020E949F190895E8EDF0E080818E7F08
:1033F00080831092E20008951092DA001092E100AA
:1034000008951F920F920FB60F9211242F933F939E
:103410004F935F936F937F938F939F93AF93BF93DC
:10342000EF93FF938091E10082FF0BC08091E20057
:1034300082FF07C08091E1008B7F8093E1000E94B2
:10344000641C8091DA0080FF19C08091D80080FF51
:1034500015C08091DA008E7F8093DA008091D900C8
:1034600080FF94C080E189BD82E189BD09B400FE7E
:10347000FDCF81E080932A020E9449168091E100ED
:1034800080FF19C08091E20080FF15C08091E200AA
:103490008E7F8093E2008091E20080618093E20061
:1034A0008091D80080628093D80019BC85E0809319
:1034B0002A020E945D168091E10084FF29C080915C
:1034C000E20084FF25C080E189BD82E189BD09B4A5
:1034D00000FEFDCF8091D8008F7D8093D800809131
:1034E000E1008F7E8093E1008091E2008F7E8093E7
:1034F000E2008091E20081608093E20080912602E8
:10350000882309F449C084E080932A020E94661649
:103510008091E10083FF29C08091E20083FF25C0F4
:103520008091E100877F8093E10082E080932A020E
:10353000109226028091E1008E7F8093E1008091BD
:10354000E2008E7F8093E2008091E20080618093B0
:10355000E20042E060E080E00E9401198091F0000A
:1035600088608093F0000E945A16FF91EF91BF91FE
:10357000AF919F918F917F916F915F914F913F910B
:103580002F910F900FBE0F901F90189519BC10929D
:103590002A020E94571672CF8091E30087FF02C073
:1035A00083E0B2CF81E0B0CF1F920F920FB60F929F
:1035B0001124FF920F931F932F933F934F935F9389
:1035C0006F937F938F939F93AF93BF93CF93DF932B
:1035D000EF93FF9309EE10E0F8018081C091EC00B9
:1035E000C795CC27C7958F70FC2EF82A1082C0EFA4
:1035F000D0E08881877F888378940E941D1BF80122
:103600001082888188608883CF2DCF70C083FF911E
:10361000EF91DF91CF91BF91AF919F918F917F916A
:103620006F915F914F913F912F911F910F91FF905B
:103630000F900FBE0F901F901895AAE2B0E0E3E242
:10364000FBE10C94A81C8BE292E0FC010196209116
:10365000F100208322E083339207B9F70E94861697
:103660008091E80083FF38C080912B0290912C025A
:103670009A3090F5E92FF0E0EA56F24E0C94931C44
:10368000803889F0823841F580912F028F70873021
:1036900018F58093E9008091EB0085FB882780F97D
:1036A0001092E90006C080912702909128029111A2
:1036B00082609091E800977F9093E8008093F100FA
:1036C0001092F1008091E8008E7723C0811116C01E
:1036D00080912D02813011F18091E80083FF0AC0B2
:1036E0008091E800877F8093E8008091EB00806202
:1036F0008093EB00AA96E3E00C94C41C823061F73F
:1037000080912D02882389F01092E9008091E800D1
:10371000877F8093E8000E943519DECF81E09330E7
:1037200009F080E080932802EFCF80912F028F7004
:103730002FEF280F263080F68093E9002091EB00D0
:1037400020FFE2CF933031F48091EB0080628093D0
:10375000EB00DACF9091EB0090619093EB0021E0C9
:1037600030E0A90102C0440F551F8A95E2F740934B
:10377000EA001092EA008091EB008860E8CF8111A6
:10378000ABCF10912D021F778091E3008078812BC1
:103790008093E3008091E800877F8093E8000E9497
:1037A00035198091E80080FFFCCF8091E3008068AC
:1037B0008093E30083E0111101C082E080932A022C
:1037C0008BCF8058823008F087CF80912D02909166
:1037D0002E028C3D53E0950799F583E08A838AE2B7
:1037E00089834FB7F894DE01139620E03EE051E262
:1037F000E32FF0E050935700849120FF03C082959F
:103800008F703F5F8F708A30C8F0895C90E08D9335
:103810009D932F5F243161F74FBF8091E800877F30
:103820008093E8006AE270E0CE0101960E944C1895
:103830008091E8008B778093E8004ECF805DE6CFE3
:1038400060912F0270913002AE014F5F5F4F0E9476
:103850008617BC01892B09F43FCF8091E800877F50
:103860008093E80089819A810E94A618E1CF803870
:1038700009F032CF8091E800877F8093E800809143
:1038800026028093F1001ECF811126CF90912D0248
:10389000923008F021CF8091E800877F8093E80084
:1038A000909326020E94351980912602882331F0D8
:1038B00084E080932A020E9471160ECF8091E3006B
:1038C00087FDF6CF81E0F5CF0895CF9380912A024E
:1038D000882399F08091E900C091EC00C795CC272E
:1038E000C7958F70C82B1092E9008091E80083FD86
:1038F0000E941D1BCF70C093E900CF91089597FBE4
:10390000072E16F4009407D077FD09D00E94D01C32
:1039100007FC05D03EF4909581959F4F08957095D2
:1039200061957F4F0895EE0FFF1F0590F491E02DF4
:1039300009942F923F924F925F926F927F928F9253
:103940009F92AF92BF92CF92DF92EF92FF920F932E
:103950001F93CF93DF93CDB7DEB7CA1BDB0B0FB638
:10396000F894DEBF0FBECDBF09942A8839884888F5
:103970005F846E847D848C849B84AA84B984C8848B
:10398000DF80EE80FD800C811B81AA81B981CE0F82
:10399000D11D0FB6F894DEBF0FBECDBFED01089567
:1039A000AA1BBB1B51E107C0AA1FBB1FA617B70765
:1039B00010F0A61BB70B881F991F5A95A9F7809581
:1039C0009095BC01CD010895FB01DC0104C08D91EF
:1039D0000190801921F441505040C8F7881B990B81
:1039E0000895FB01DC0102C001900D92415050404E
:1039F000D8F70895F999FECF92BD81BDF89A99271D
:103A000080B50895A8E1B0E042E050E00C943E1D7E
:103A1000DC01A40FB51F4150504048F0CB01840F8A
:103A2000951F2E910E94191D41505040D0F70895C6
:103A3000262FF999FECF92BD81BDF89A019700B467
:103A4000021639F01FBA20BD0FB6F894FA9AF99A07
:103A50000FBE08950396272F0E94191D0E94181D5E
:103A6000252F0E94191D242F0C94191D0196272F14
:103A70000E94191D0C94181DDC01CB01FC01F99961
:103A8000FECF06C0F2BDE1BDF89A319600B40D92AA
:103A900041505040B8F70895F894FFCF7E037E035D
:103AA000C503C5032A044704AD03AD034C04C30496
:103AB000D404D404221096102A10F40FF80F2E10FC
:103AC000FC0F32103E1008108F100C104210101016
:103AD00046106E1014104A1075101A10501058101D
:103AE0000010361004103A101E10541064107E108E
:103AF0008D10EE0F26109D10411147114A115011E3
:103B00006511651165116511651165116511651105
:103B1000531158115C116211731179117D11B21397
:103B2000B813A213AC13BE13C413CA13401B661BF5
:103B30006C1B661B6C1BBF1BE11B6C1B371C441CE6
:103B4000E201280850011E0A1401FC153216FF1567
:103B50002B16241601E200E900EA00B500B600B712
:103B600000CD008301CC008A01920194012102233F
:103B70000224022502260227022A02B300B4006FA3
:103B80000070009F01CB019F02A002E200E900EA61
:103B900000B500B600B700CD008301CC008A0192C9
:103BA0000194012102230224022502260227022A6F
:103BB00002B300B4006F0070009F01CB019F02A010
:063BC00002F4F63132347C
:00000001FF
